:020000040000FA
:020000002528B1
:080008008F00030803138312AB
:100010008E0004088C000A088D008A010B19112833
:100020001C280B11063081008B018B168B171708CB
:10003000031D970344201C280D088A000C08840027
:100040000E0883008F0E0F0E0900832076200530E6
:100050007E20262882073F3406345B344F346634D2
:100060006D347D3407347F34673477347C345834CE
:100070005E34793471348207013402340434083434
:100080001034203440348034140884000310840C6D
:1000900010308407000898001418980E18080F39BB
:1000A0002A20950014083B2096005D201408031DAB
:1000B0005B28083094009403080008308510161C53
:1000C0006228851405140510960CFF3E031D5E285A
:1000D00008308510151C6D28851405140510950C25
:1000E000FF3E031D6928051505110800900F080043
:1000F000910F0800920F0800930A08009700170854
:10010000031D7F2808008B018B168316850186014D
:100110008101013081048312103084000430800199
:10012000FF3E03199528840A8F2806308100073086
:10013000940005110510950196015D208B170800AC
:084000000100020003000400AE
:02400E00F13F80
:1042000043006F0070007900720069006700680069
:104210007400200032003000300032002C002000FA
:10422000540075006E006400720061005700610068
:1042300072006500200049006E0063002E0020001F
:10424000200041006C006C002000520069006700F3
:104250006800740073002000520065007300650060
:0A42600072007600650064002E0075
:00000001FF
